:04000000F8EF0DF018
:08000800046ED8CF05F0E0CF33
:1000100006F00001E9CF0CF0EACF07F0E1CF08F0DD
:10002000E2CF09F0D9CF0AF0DACF0BF0F3CF12F01C
:10003000F4CF13F0FACF14F0F5CF15F0F6CF16F099
:10004000F7CF17F000C00EF001C00FF002C010F0A3
:1000500003C011F09DA030EF00F09EB007EF02F05A
:100060009DA236EF00F09EB29AEF01F0F2A63CEFAF
:1000700000F0F2B0F1EF00F09DAA42EF00F09EBA5E
:1000800091EF02F09DA848EF00F09EB815EF03F045
:100090000EC000F00FC001F010C002F011C003F05C
:1000A0000CC0E9FF07C0EAFF078E08C0E1FF09C0E6
:1000B000E2FF0AC0D9FF0BC0DAFF12C0F3FF13C082
:1000C000F4FF14C0FAFF15C0F5FF16C0F6FF17C005
:1000D000F7FF045006C0E0FF05C0D8FF1000F76A24
:1000E000EE0FF66E000EF7220900F55012003437BD
:1000F000313037300000F76A060FF66E010EF72236
:100100000900F55012003030303232320000F76A08
:100110001E0FF66E010EF7220900F5501200303066
:100120003031313100007374617475733A5B7469F6
:100130006C6C5D007374617475733A5B6672E56E26
:100140005D00202020200000202020200000206FC3
:100150006B20000020202020000020202B20000009
:100160002070E5200000206F6B2000002056E42066
:10017000000020202020000020202D2000006E659F
:100180006A002062797400002048F6200000416E69
:100190006765206CF673656E6F726400016A026AAF
:1001A000006A036A01014F5102E14E5118E0100E3E
:1001B000506FD8904C374D37003603364F51035CA3
:1001C00002E14E51005C07E34E51005ED8A00306E9
:1001D0004F51035ED88001360236502FEAD7000116
:1001E000120081BE01D02D8081BC01D02D822D5006
:1001F0000F0BF00F0DE2100F5CEF01F009D08551ED
:10020000D8B48607850704D0852BD8B4862B00D0B8
:100210002D362D36FC0E2D1681BA01D03A8081B8CC
:1002200001D03A823A500F0BF00F08E2100F79EF2D
:1002300001F004D03D0602D03D2A00D03A363A36CD
:10024000FC0E3A163C503D5C02E18294829682BAE2
:1002500030D081BE2ED081BC2CD086C0C0F085C0ED
:10026000BFF0C0C04DF1BFC04CF101014F6B6DC07C
:100270004EF1000193DF00C0BFF003C0C0F0BF51DA
:10028000C01117E0D8906D30C05307E1BF5D05E2A3
:10029000BF51855FC051865B0AD0BF516D5C006E57
:1002A000000EC055036E0050852703508623C06B97
:1002B000BF6BF29048EF00F0E824F76AF736D30FEF
:1002C000F66E020EF7220A00F550FA6E0800F5509D
:1002D000F96EFC01FE01080210020802FC01100286
:1002E000FE01FE011002FC01080210020802FE01DC
:1002F000FC01E824F76AF7360D0FF66E030EF722BD
:100300000A00F550FA6E0800F550F96E3202340218
:1003100038023C02380232023C02340234023C020F
:10032000320238023C023802340232029EA8FED762
:10033000AD6E1200CA94ABA808D0AB98818463500C
:10034000F5DF010E256E9D8802D08194AB889E92C8
:1003500048EF00F00101516B4DC150F1F250006EB9
:10036000F29EAA6A4CC1A9FF50C1A8FFA69CA69EF6
:10037000A6840F01550EA76EAA0EA76EA682A6B27E
:10038000FED7A6940050F21201014F2D1AD04EC193
:1003900051F14C2BF250006EF29EAA6A4CC1A9FF9B
:1003A00051C1A8FFA69CA69EA6840F01550EA76E5C
:1003B000AA0EA76EA682A6B2FED7A6940050F2128D
:1003C000010100011200F29CF29EF2BEFDD7819461
:1003D0001B0E01014C6FBCC04EF1BBC04DF1010EB4
:1003E0004F6F0001B7DFFFD715EF02F08194AB88A4
:1003F000656A190E6A6EBE6BBD6B206AC26BC16BFB
:100400001D961E9CC46BC80EC36F746A1200FB0E4F
:10041000CF6E800ECE6E040081A008D04C2A4C50C6
:10042000040803E21EA201D0CED701D04C6A6A5262
:1004300002E06A060AD0BD51BE1107E1655205E02F
:10044000BE6BFA0EBD6F6B6A796A242A24500A08C3
:100450002BE1246ABD51BE1127E0696A6950030887
:1004600018E3036A6950700FE96E000E0320EA6E0C
:10047000EF520DE0036A6950700FE96E000E032021
:10048000EA6EEF6A6950100DF3CF22F002D0692AAC
:10049000E5D7256AAB988184010E48DF79501D08A5
:1004A00001E2A4DF792A9D88282A2850140802E155
:1004B000286A1D82272A2750640802E1276A1D80C6
:1004C0009E9048EF00F09EAAFED7ABCF1CF0AECFB7
:1004D00001F01CA202D0AB98AB8892EF02F01E8C08
:1004E000C46BC36B7850010A07E0030A0AE0010AF3
:1004F0000AE0070A0DE011D00B0EC26FB90EC16FF2
:100500000ED01E8E0CD0070EC26FD10EC16F07D059
:10051000030EC26FEA0EC16F02D0C26BC16BC2EF95
:1005200002F0D1D701C00AF1BD51BE1143E1010172
:100530000A51010A000103E0030A03E02DD0506ACA
:1005400038D05050020827E151501F0B070823E113
:100550005250040818E16B2A6B50020813E2526AE9
:100560006B6A5138786E7832070E78167850020828
:1005700002E0010E656E796A785202E0B0D702D0CF
:10058000C26BC16B01D06B6A516A190E6A6E205042
:10059000080801E0CA840DD0036A5050510FE96E7B
:1005A000000E0320EA6E0AC1EFFF5050100801E36D
:1005B000502A38D0036A36502E0FE96E000E032001
:1005C000EA6E0AC1EFFF362A365008082BE1366A78
:1005D000365006080BE3036A36502E0FE96E000E04
:1005E0000320EA6EEF503726362AF2D73550375CB3
:1005F00019E1795201E079062EC026F026500F0B42
:100600006E6E1D866E5204E0BE6BFA0EBD6F0AD090
:10061000BD51D8B4BE07BD07BD51BE1102E0655241
:1006200001E1E4DE9E9A48EF00F0BD51BE112CE1DD
:10063000010E255CFB0F27E2050F89EF03F06450E4
:1006400075DE252A20D0655071DE252A1CD0665023
:100650006DDE252A18D0675069DE252A14D09D98B2
:10066000686A696A695004080BE3036A6950630F9A
:10067000E96E000E0320EA6EEF506826692AF2D771
:10068000685054DECA8442D0255007E0010A09E0D0
:10069000030A10E0010A1EE038D0840E47DE252A46
:1006A00035D0030E222401014C6F4C5100013EDE77
:1006B000252A2CD02250222A036AC90FE96E000E87
:1006C0000320EA6EEFCF4CF101014C5100012EDE08
:1006D000252A1CD022500F0B0FE02250222A036A39
:1006E000C90FE96E000E0320EA6EEFCF4CF1010155
:1006F0004C5100011BDE08D09D98020E17DE3F0E04
:100700002216366A376ACA8401D0226A9E9848EF58
:1007100000F0E824F76AF7362D0FF66E070EF72281
:100720000A00F550FA6E0800F550F96E3E064606CE
:100730004E0656065E06D67672696720696E666F4B
:100740000000262066756E6B74696F6E657200001E
:1007500054696C6C62616B612074696C6C006D61D2
:10076000737465722073747972656E6865740000C5
:100770004E7920736C616E672D0070E56CE46767DD
:100780006E696E6700006CE467655B4F4B5D00004F
:100790006CE467655B46454C5D005374617274613F
:1007A000206F6D00736C616E67656E686574000024
:1007B0004D656E7920256C75000074657374612039
:1007C0004F70746F380074696C6C00006672E56E6F
:1007D000000053746174757320696E67202620755C
:1007E000746700004BF672206C65646172650000EE
:1007F0006D616E75656C6C7400004769762074726B
:10080000756D6D6120667200696E672E3120706CA7
:10081000696E74203200476976207472756D6D615F
:1008200020626100696E672E3220706C696E7420E0
:100830003500476976206C65646172652068F60052
:10084000696E672E3320706C696E742038004769BA
:1008500076206C65646172652076E400696E672EAF
:100860003420706C696E742031310000496E64650B
:10087000786769760000696E672E3520706C696E46
:100880007420313400004F7074696F6E0000696E1F
:10089000672E3620706C696E7420313700004F70FF
:1008A00074696F6E0000696E672E3720706C696E18
:1008B000742032340000496E7374E46C6C6E696E9F
:1008C000676172004279742074696C6C20736C618A
:1008D0006E6700005B25326C755D6D6D2E005B25CB
:1008E000326C755D6D6D2E00557476E4786C696EB2
:1008F000670050613A20383120762F733A202575F1
:100900002E2575004E61766469616D6574657200AF
:1009100050613A203833206D6D3A25346C750000F3
:10092000536C616E676469616D65746572005061D6
:100930003A203835206D6D3A25336C7500005061D2
:1009400072616D657465725B2533755D0000506181
:100950003A253375000056E47264655B25356C7585
:100960005D004772756E64696E7374E46C6C6E2E14
:1009700000006D6564203333302072756C6C650047
:100980004772756E64696E7374E46C6C6E2E000051
:100990006D6564203239302072756C6C65004F7063
:1009A00074696F6E00004CF673656E6F72640000C0
:1009B0003234652E312E312E30352E630000323424
:1009C0002D6A616E2D32300031393A31313A353885
:1009D000000046656C206CF673656E6F72640000F3
:1009E0007472756D6D613A25346C75002D2D2D2D49
:1009F0002D2D2D2D2D2D2D2D2D2D2D2D00006B6F01
:100A00006C763A25327500002D2D2D2D2D2D2D2D96
:100A10002D2D2D2D2D2D2D2D00000101336BF2CF0D
:100A200034F1F29EAA6A2EC1A9FFA69CA69EA680BA
:100A3000A85034BFF28E326F2F2D18D02E2BF2CF4C
:100A400034F1F29EAA6A2EC1A9FFA69CA69EA6809A
:100A5000A85034BFF28E336F33C131F132C130F15F
:100A600030C101F031C102F008D003D0316B32C186
:100A700030F130C101F031C102F00001120001017A
:100A8000456B466B010E476FDA6AD96A4A6F3D0EB5
:100A9000496F010EEA6E410EE96E4AC1E2FF49C19B
:100AA000E1FF47C148F1D890E550EE02F3504523ED
:100AB000F4504623482FF7D745C1DEFF46C145F124
:100AC000466BD8B0462B492BD8B44A2B472B4751FD
:100AD0000508DFE100011200D8B204D0010EEA6E71
:100AE000470EE96E006A016A026A036A0101476BF8
:100AF000486B496B4A6B46514511441143112CE038
:100B0000200E4B6FD8903F37403741374237473739
:100B1000483749374A3746514A5D08E14551495DF2
:100B200005E14451485D02E14351475D0FE3435104
:100B3000475F4451D8A0443D485F4551D8A0453D4A
:100B4000495F4651D8A0463D4A5FD88000360136FD
:100B5000023603364B2FD6D747C1EFFF48C1ECFF13
:100B600049C1ECFF4AC1ECFF0001120001012D5107
:100B70002F03F3CF01F0F4CF00F03003F350002641
:100B80002E512F03F3500020026E00011200510E6F
:100B90003B2401012D6F2E6F010E2F6F00013DDFF1
:100BA00001011E6B1D6B02C01CF101C01BF1530E35
:100BB0003B242D6F2E6F010E2F6F00012EDF0101E0
:100BC000226B216B02C020F101C01FF1550E3B24A6
:100BD0002D6F2E6F010E2F6F00011FDF0101266B9D
:100BE000256B02C024F101C023F1590E2E6F2F6B2B
:100BF000000113DF01C02BF101011B5307E11C535E
:100C000005E11D5303E11E53D8B4ADD11F5307E1D5
:100C1000205305E1215303E12253D8B4A4D1235337
:100C200007E1245305E1255303E12653D8B49BD1B2
:100C30002B53D8B498D104001EC140F11DC13FF11F
:100C40001CC13EF11BC13DF1446B436B426B2BC198
:100C500041F1000114DF03C030F102C02FF101C0E7
:100C60002EF100C02DF101012D372E372F373037EF
:100C70002D372E372F373037FC0E2D17D89230C135
:100C800042F12FC141F12EC140F12DC13FF1466B20
:100C9000456B446B0A0E436F00011EDF01C088F0F4
:100CA00000C087F088C02EF187C02DF10101306BA4
:100CB000640E2F6F00015ADF02C02EF101C02DF12A
:100CC000036A4AC02FF1010103C030F1196AF2BE74
:100CD000198EF29E02C04DF101C04CF103C04FF1DC
:100CE0004AC04EF10001CEEC00F019BEF28E02C0F7
:100CF000B2F001C0B1F0D8921EC142F11DC141F164
:100D00001CC140F11BC13FF10101466B456B446BB7
:100D10000A0E436F0001E0DE010E01010024276F7F
:100D2000000E0120286F000E0220296F000E032004
:100D30002A6F2AC140F129C13FF128C13EF127C1E4
:100D40003DF1446B436B426B2BC141F1000197DED7
:100D500003C030F102C02FF101C02EF100C02DF10F
:100D600001010034006E0134016E0234026E03345E
:100D7000036E0036013602360336FC0E001600C044
:100D800089F0000101C08AF001012C6B2C510E0882
:100D9000D8A0E9D00400D8902C35036A910FE96EF1
:100DA000000E0320EA6E23511F252F6F24512021AE
:100DB000306F25512121316F26512221326FEACF28
:100DC00034F1E9CF33F1406B3F6B3E6B2CC13DF109
:100DD00026C144F125C143F124C142F123C141F1AF
:100DE00000014DDE34C1EAFF33C1E9FF03C038F131
:100DF00002C037F101C036F100C035F1EACF3AF157
:100E0000E9CF39F103C040F102C03FF101C03EF12A
:100E100000C03DF10101446B436B426BB90E416F61
:100E200000012DDE3AC1EAFF39C1E9FF03C038F104
:100E300002C037F101C036F100C035F1EACF3CF114
:100E4000E9CF3BF1D89203C042F102C041F101C0A9
:100E500040F100C03FF10101466B456B446B640EED
:100E6000436F000139DE3CC1EAFF3BC1E9FF00509E
:100E700001012F2701503023025031230350322328
:100E8000EACF36F1E9CF35F132C140F131C13FF15E
:100E900030C13EF12FC13DF1446B436B010E426FF7
:100EA0003A0E416F0001EBDD36C1EAFF35C1E9FFC3
:100EB00003C032F102C031F101C030F100C02FF1A6
:100EC000EACF38F1E9CF37F103C040F102C03FF17A
:100ED00001C03EF100C03DF12AC144F129C143F1F6
:100EE00028C142F127C141F1CADD38C1EAFF37C14B
:100EF000E9FF03C032F102C031F101C030F100C09E
:100F00002FF1EACF3EF1E9CF3DF1D89203C042F193
:100F100002C041F101C040F100C03FF10101466B48
:100F2000456B270E446F100E436F0001D5DD3EC1A7
:100F3000EAFF3DC1E9FF00C0EFFF01C0ECFFD89020
:100F400001012C35036A910FE96E000E0320EA6E51
:100F5000ECCF03F0ED52EF500001832703508423C0
:100F600001012C2B13D70001B1EF0EF0010EEA6E38
:100F70001C0EE96EEF500EE0010E016E006A002EAD
:100F8000FED7012EFBD7300E006E002EFED700D00C
:100F9000EF2EF2D7120001011B6B1B513F080BE330
:100FA000036A1B51C90FE96E000E0320EA6E200E82
:100FB000EF6E1B2BF2D71B6B1B5103080BE3036A6D
:100FC0001B51700FE96E000E0320EA6E010EEF6EEA
:100FD0001B2BF2D7216A00014DEF0FF001011E51CA
:100FE000100DF3501F25216E3F0E21160001120037
:100FF0000101265324E0036A2150C90FE96E000E57
:101000000320EA6E2651EF5C16E0036A2150C90FF7
:10101000E96E000E0320EA6E26C1EFFF2138006E54
:101020000F0E00160050036A700FE96E000E0320C9
:10103000EA6E010EEF6E21503E0801E3212A000105
:1010400012000900F5520CE0F6CF1EF1F7CF1FF1A8
:10105000F5CF26F1CDDF1EC1F6FF1FC1F7FFF1D797
:101060001200036A2150C90FE96E000E0320EA6ED8
:10107000EF50200816E0036A2150C90FE96E000EF8
:101080000320EA6E200EEF6E2138006E0F0E001660
:101090000050036A700FE96E000E0320EA6E010E25
:1010A000EF6E212A21500F0BDCE11200006A016A69
:1010B00001011E51D8901FB10026003201321FB32A
:1010C0000026003201321FB50026003201321FB760
:1010D0000026003201321FB90026003201321FBB48
:1010E0000026003201321FBD0026003201321FBF30
:1010F00000260032013200011200030E01011E6FB2
:101100001F6B00016BDF01011E6B1C51F00B1F6F89
:101110001E530AE11F5308E1420EF66E010EF76EF0
:1011200000018FDF1DD001011E6B1C51F00B1F6FE2
:101130001E5317E11F51100814E1200E266F000105
:1011400057DF7F0E0101266F000152DF200E0101E3
:10115000266F00014DDF200E0101266F000148DFE0
:1011600001011E6B1C510F0B1F6F1E530AE11F5311
:1011700008E1480EF66E010EF76E000162DF2DD019
:1011800001011E6B1C510F0B1F6F1E5317E11F2D0A
:1011900015D0200E266F00012BDF7E0E0101266F79
:1011A000000126DF200E0101266F000121DF200E45
:1011B0000101266F00011CDF10D001011E6B1C51C4
:1011C0000F0B1F6F1E530AE11F51040807E14E0E5B
:1011D000F66E010EF76E000134DF01011B51F00BBA
:1011E0001E6F1F6B1E530AE11F5308E1540EF66E6B
:1011F000010EF76E000125DF61D001011B51F00BDC
:101200001E6F1F6B1E51100817E11F5315E1200EB2
:10121000266F0001EDDE200E0101266F0001E8DEE1
:10122000060E0101266F0001E3DE200E0101266F8C
:101230000001DEDE43D001011B51F00B1E6F1F6B5E
:101240001E5120080AE11F5308E15A0EF66E010EE6
:10125000F76E0001F6DE32D001011B51F00B1E6F5C
:101260001F6B1E5130080AE11F5308E1600EF66E35
:10127000010EF76E0001E5DE21D001011B51F00BDC
:101280001E6F1F6B1E5140080AE11F5308E1660ED6
:10129000F66E010EF76E0001D4DE10D001011B5175
:1012A000F00B1E6F1F6B1E51600809E11F5307E111
:1012B0006C0EF66E010EF76E0001C3DE01011B51CC
:1012C0000F0B1E6F1F6B1E530AE11F5308E1720EB6
:1012D000F66E010EF76E0001B4DE60D001011B5105
:1012E0000F0B1E6F1F6B1E2D17D01F5315E1200E05
:1012F000266F00017DDE200E0101266F000178DEE1
:10130000050E0101266F000173DE200E0101266F1C
:1013100000016EDE43D001011B510F0B1E6F1F6BCE
:101320001E5102080AE11F5308E1780EF66E010E05
:10133000F76E000186DE32D001011B510F0B1E6FCC
:101340001F6B1E5103080AE11F5308E17E0EF66E63
:10135000010EF76E000175DE21D001011B510F0B4C
:101360001E6F1F6B1E5105080AE11F5308E1820E14
:10137000F66E010EF76E000164DE10D001011B5104
:101380000F0B1E6F1F6B1E51060809E11F5307E16B
:10139000880EF66E010EF76E000153DE01011EA8E5
:1013A00008D06E5205E11E980001C66BC56B0101A5
:1013B0005CD16E52D8B444D10001C46BC36B01013F
:1013C0001D5304E11E88010E6F6E33D00001C6C0AC
:1013D0001FF1C551C52BD8B4C62B01011E6F1E537A
:1013E00005E11F5303E1010E6F6E23D00001C653C8
:1013F00003E1C55128080BE201011D510208D8B4D0
:1014000002D0000104D0140E6F6E13D00001C65339
:1014100003E1C551140803E2050E6F6E09D0C653EF
:1014200003E1C551070803E2010E6F6E01D06F6A38
:1014300001011E6B1C51F00B1F6F1E5311E11F5158
:1014400010080EE16E5008080BE10001C151D8B43C
:10145000C207C1071E88000E016E0AD1EFD001013C
:101460001E6B1C510F0B1F6F1E530FE11F2D0DD054
:101470006E5004080AE10001C12BD8B4C22B1E88AB
:10148000000E016EF5D0DAD001011E6B1C510F0B5E
:101490001F6F1E5310E11F5104080DE16E50040828
:1014A0000AE10001C12BD8B4C22B1E88000E016EC8
:1014B000DFD0C4D001011B51F00B1E6F1F6B1E51FA
:1014C00010080FE11F530DE16E5002080AE1E80E0B
:1014D0000001C15F030EC25B000E016EC9D0AED029
:1014E00001011B510F0B1E6F1F6B1E2D0ED01F53C2
:1014F0000CE16E2C0AD0E80E0001C127030EC223B6
:10150000000E016EB5D09AD001011B51F00B1E6F79
:101510001F6B1E5120080BE11F5309E16E5002089A
:1015200006E16FC001F00001A3D088D001011B517A
:101530000F0B1E6F1F6B1E5102080DE11F530BE1B5
:101540006E2C09D06FC01EF11F690001AFDD015084
:101550008FD074D001011B51F00B1E6F1F6B1E51F9
:1015600030080BE11F5309E16E50020806E16FC01D
:1015700001F000017DD062D001011B510F0B1E6FE5
:101580001F6B1E5103080DE11F530BE16E2C09D098
:101590006FC01EF11F69000189DD015069D04ED076
:1015A00001011B51F00B1E6F1F6B1E5140080BE118
:1015B0001F5309E16E50020806E16FC001F00001FF
:1015C00057D03CD001011B510F0B1E6F1F6B1E51DA
:1015D00005080DE11F530BE16E2C09D06FC01EF101
:1015E0001F69000163DD015043D028D001011B5168
:1015F000F00B1E6F1F6B1E5160080BE11F5309E1BA
:101600006E50020806E1FF0E016E000131D016D0C7
:1016100001011B510F0B1E6F1F6B1E5106080AE1C3
:101620001F5308E16E2C06D0010E016E000120D080
:1016300005D00101000E016E00011AD015D0010184
:101640000001C66BC56BC4C01FF1C351C32BD8B416
:10165000C42B01011E6F1F5303E11E51C80805E290
:101660000001C26BC16B1E9C0101000E016E0001E6
:10167000120082B402D082A605D03E503D5C02E149
:101680003F2A03D03F6A3DC03EF048503F5C0FE325
:101690001EB60CD082A608D03D50180805E38296ED
:1016A0000A0E3D6E3C6E01D01D8C01D01D8C1200C7
:1016B0001E863F6A1D9C3D6A040E3C6E82841D920C
:1016C0000F0E286E1DA202D01D92D3DF82A402D07D
:1016D0001DACF8D7320E01011C6F000147DC82946B
:1016E000320E01011C6F000141DC140E4A243D6ED4
:1016F0003C6A82861D920F0E286E1D9C1DA202D090
:101700001D92B7DF82A602D01DACF8D7320E0101C0
:101710001C6F00012BDC8296320E01011C6F000150
:1017200025DC3F6A1D9C1E9612000900F6CF1EF1B3
:10173000F7CF1FF1F5CF26F15BDC1EC1F6FF1FC10D
:10174000F7FF01011D2F01D002D00001EED70001EB
:101750001200EACF25F1E9CF24F101011E39F00989
:10176000206F2027E20F216F320F236F1E510F0BC6
:10177000212721272327E90F226F222722271D391E
:101780000F0B2227232722372337231F23371D51EF
:101790000F0B23272037070E1F6F0A0E2207232760
:1017A000FDE321072227FDE320072127FDE31F0793
:1017B0002027FDE3010EEA6E1F0EE96E070E2415C9
:1017C000249DE926000EEA22E950230803E1EA2CD1
:1017D00001D0248DEF50006E08E124BD06D024B95D
:1017E00016D024B702D0200E03D024872499300EBF
:1017F0000026EACF1EF1E9CF1DF100C026F100015D
:10180000F8EC07F01EC1EAFF1DC1E9FF0101EE502F
:1018100024ADDAD70001120001012051016A1F5DD9
:1018200003E21FC100F00CD0006A080E216F1F37C1
:1018300000362051005CD8B0006E0136212FF7D75A
:101840000001120001501DC11FF1640E0101206F43
:101850000001E2DF00C01DF10150300E08E101017E
:101860001EA310D01EB70ED01EB9200E04D0010149
:101870001E971E991E81012601C026F10001F8EC79
:1018800007F001011DC11FF10A0E206F0001C4DF26
:1018900000C01DF10150300E08E101011EB70BD050
:1018A0001EA109D01EB9200E0001012601C026F19B
:1018B000F8EC07F00101300E1D271DC126F10001D3
:1018C000F8EC07F0120001011C911B51010A000104
:1018D00011E0030A15E00B0A19E0030A1DE0010AF2
:1018E00021E0070A25E0010A29E0030A2DE0010AA8
:1018F00031E036D082A403D001011C81000130D038
:1019000082A603D001011C8100012AD081BE03D030
:1019100001011C81000124D081BC03D001011C8184
:1019200000011ED081BA03D001011C81000118D032
:1019300081B803D001011C81000112D082B803D00C
:1019400001011C8100010CD082BA03D001011C816D
:10195000000106D081B203D001011C81000100D03A
:1019600001011CA109D0260EF66E010EF76E0001D2
:1019700021EC08F008D00101340EF66E010EF76E6E
:10198000000121EC08F0120001011E6B1F6B000129
:10199000EEEC07F08E0EF66E010EF76E21EC08F0FD
:1019A00031EC08F0010E01011E6F1F6B0001EEEC1F
:1019B00007F0010E696E695006080DE3036A69506D
:1019C0000B0FE96E010E0320EA6EEFCF26F1F8EC63
:1019D00007F0692AF0D731EC08F0020E01011E6F02
:1019E0001F6B0001EEEC07F0010E696E69500608EE
:1019F0001AE3880EC15D006E130EC259036E0050CB
:101A0000695C09E1035207E12D0E0101266F000117
:101A1000F8EC07F006D0200E0101266F0001F8EC6B
:101A200007F0692AE3D731EC08F0120001011F53D7
:101A300002E1205344E01CC103F01BC1E9FF03C0D5
:101A4000EAFFEFCF21F11EC103F01DC1E9FF03C082
:101A5000EAFFEF50215D17E01CC103F01BC1E9FF55
:101A600003C0EAFFEFCF21F11EC103F01DC1E9FF62
:101A700003C0EAFFEF50215D02E2FF0E01D0010E2C
:101A8000016E1FD00BD01CC103F01BC1E9FF03C0C6
:101A9000EAFFEF5203E1000E016E13D01CC103F008
:101AA0001B511B2BD8B41C2B1EC103F01D511D2B29
:101AB000D8B41E2B1F51D8B420071F07B8D7000E6B
:101AC000016E00011200196AF2BE198EF29E86C0E4
:101AD0004DF185C04CF18AC04FF189C04EF1CEEC7A
:101AE00000F019BEF28E01C02CF0906B8F6B0101DB
:101AF0001B6B2C501B5D13E2D8901B35036A910FB2
:101B0000E96E000E0320EA6EECCF03F0ED52EF50C9
:101B100000018F270350902301011B2BEAD7D89097
:101B20002C34036A910FE96E000E0320EA6EECCFAD
:101B30001DF1ED52EFCF1CF11E6B1F6B8AC02EF111
:101B400089C02DF1306B2CC02FF10001B6EC05F0EF
:101B50000150855D006E02508659036E00C020F171
:101B60000101216FEACF23F1E9CF22F11FC140F13A
:101B70001EC13FF11DC13EF11CC13DF1446B436BE1
:101B8000426F00C041F100013FEC05F023C1EAFFC4
:101B900022C1E9FF03C01FF102C01EF101C01DF107
:101BA00000C01CF1EACF21F1E9CF20F1D89203C0A7
:101BB00042F102C041F101C040F100C03FF101011A
:101BC000466B456B8AC044F189C043F100016CEC5F
:101BD00005F021C1EAFF20C1E9FF8F510101002476
:101BE0000001836F9051010101200001846F1200F8
:101BF000F86AD09E078E7E0E006E100E016E020EE9
:101C0000E96E000EEA6EEE6A0400002EFCD7012E8B
:101C1000FAD71C6AB896020EAF6EA20EAC6E900E8A
:101C2000AB6E01011A6B196BC150C00B0F09C16E6D
:101C3000070EB46E1A6A1B6A000E926EF30E936E54
:101C4000B00E946E8294829682928290B40E2A6E26
:101C5000D180590E2E6F2F6B00010DEC05F002C0E4
:101C60001CF101010134026E1C35036E023603368D
:101C7000FC0E021602C06DF00A0E2E6F2F6B0001D3
:101C80000DEC05F00150021003E0640E3B6E01D034
:101C90003B6A3BC02EF101012F6B00010DEC05F0FA
:101CA00001C040F0010E3B2401011B6F2E6F2F6B12
:101CB00000010DEC05F001C041F0020E3B240101D2
:101CC0001B6F2E6F2F6B00010DEC05F001C042F071
:101CD000030E3B2401011B6F2E6F2F6B00010DECD7
:101CE00005F001C043F0040E3B2401011B6F2E6F71
:101CF0002F6B00010DEC05F001C044F0050E3B24F4
:101D000001011B6F2E6F2F6B00010DEC05F001C060
:101D100045F0060E3B2401011B6F2E6F2F6B000157
:101D20000DEC05F001C046F0070E3B2401011B6FCE
:101D30002E6F2F6B00010DEC05F001C047F0060E71
:101D4000486E090E3B2401011B6F2E6F2F6B0001A3
:101D50000DEC05F001C04AF00400190E6A6EC7EFE1
:101D600005F004001B0E01012E6F010E2F6F000104
:101D70000DEC05F002C086F001C085F0640E010193
:101D80001C6F0001B6EC07F081BE01D02D8081BC34
:101D900001D02D822D362D36FC0E2D16196AF2BE7D
:101DA000198EF29E86C04DF185C04CF188C04FF16E
:101DB00087C04EF1CEEC00F019BEF28E02C01CF1CD
:101DC00001C01BF1010101A017D0196AF2BE198EE2
:101DD000F29E86C04DF185C04CF188C04FF187C09E
:101DE0004EF10001CEEC00F019BEF28E00C0B5F04D
:101DF00003C0B6F018D00101196AF2BE198EF29E26
:101E000086C04DF185C04CF188C04FF187C04EF1BE
:101E10000001CEEC00F019BEF28E0050875DB56F68
:101E200003508859B66FB6C02EF1B5C02DF101012F
:101E3000306B640E2F6F0001B6EC05F002C01CF190
:101E400001C01BF1196AF2BE198EF29E02C04DF15B
:101E500001C04CF1B2C04FF1B1C04EF1CEEC00F078
:101E600019BEF28E01C01BF10A0E01010124016EA0
:101E7000000E022001C03CF03CC03DF0B50ECD6E1E
:101E8000080E0509CA6EC00ECB6E9D809D82F2863B
:101E90009D8AF2120001CBEF07F00A0E01011C6FC0
:101EA0000001B6EC07F0010E855DC76F000E865984
:101EB000C86F010E855DB36F000E8659B46F010EB9
:101EC000855DB96F000E8659BA6F1D8A190E6A6E4C
:101ED000C06BBF6B6D5203E081A201D01E8E81B238
:101EE00004D0050E206E0D0E236EC151C211D8B460
:101EF0003CEF1CF01DA63CEF1CF01D96B40E2A6EA4
:101F00006E50090809E1C26BC16B206A656A1E9CAC
:101F1000C46BC80EC36F746AC1C000F0C2C003F0C6
:101F2000030EC25D04E1E80E005CD8B4FFD0030EDE
:101F3000035C04E1E90E005CD8B429D1030E035C14
:101F400004E1EA0E005CD8B461D1030E035C04E145
:101F5000EB0E005CD8B4D5D1030E035C04E1EC0EAB
:101F6000005CD8B41FD2070E035C04E1D00E005C05
:101F7000D8B464D2070E035C04E1D10E005CD8B47F
:101F800086D2070E035C04E1D20E005CD8B4EDD219
:101F9000070E035C04E1D30E005CD8B41CD3070E1B
:101FA000035C04E1D40E005CD8B44BD3070E035C91
:101FB00004E1D50E005CD8B47AD3070E035C04E1CB
:101FC000D60E005CD8B4A9D3070E035C05E1D70E8A
:101FD000005CD8B4C3EF13F0070E035C05E1D80E24
:101FE000005CD8B4F9EF13F00B0E035C05E1B80EFA
:101FF000005CD8B42FEF14F00B0E035C05E1B90EB2
:10200000005CD8B45AEF14F00B0E035C05E1BA0E75
:10201000005CD8B472EF15F00B0E035C05E1BB0E4B
:10202000005CD8B424EF16F00B0E035C05E1BC0E87
:10203000005CD8B4B3EF16F00B0E035C05E1BD0EE7
:10204000005CD8B43EEF17F00B0E035C05E1BE0E4A
:10205000005CD8B49BEF17F00B0E035C05E1BF0EDC
:10206000005CD8B456EF18F00B0E035C05E1C00E0F
:10207000005CD8B48FEF18F00B0E035C05E1C10EC5
:10208000005CD8B4C9EF18F00F0E035C05E1A00E98
:10209000005CD8B41FEF1AF0130E035C05E1880E44
:1020A000005CD8B448EF1AF0130E035C05E1890E0A
:1020B000005CD8B482EF1AF0130E035C05E18A0EBF
:1020C000005CD8B482EF1AF0130E035C05E18B0EAE
:1020D000005CD8B482EF1AF0130E035C05E18C0E9D
:1020E000005CD8B482EF1AF0130E035C05E18D0E8C
:1020F000005CD8B482EF1AF0130E035C05E18E0E7B
:10210000005CD8B4E7EF1AF0130E035C05E18F0E04
:10211000005CD8B44CEF1BF0230E035C05E1280EE5
:10212000005CD8B41FEF1CF039EF1CF001011E6BEE
:102130001F6B0001EEEC07F0360EF66E070EF76E21
:1021400021EC08F031EC08F0010E01011E6F1F6B4D
:102150000001EEEC07F0420EF66E070EF76E21EC72
:1021600008F031EC08F0020E01011E6F1F6B000138
:10217000EEEC07F031EC08F0010E01011C6F110EBE
:102180001B6F1D6B00017DEC08F03BEF1CF00101A3
:102190001E6B1F6B0001EEEC07F0500EF66E070E83
:1021A000F76E21EC08F031EC08F0010E01011E6F12
:1021B0001F6B0001EEEC07F05E0EF66E070EF76E79
:1021C00021EC08F0020E01011E6F1F6B0001EEEC06
:1021D00007F031EC08F0030E01011E6F1F6B0001C8
:1021E000EEEC07F031EC08F0110E01011C6F400E0F
:1021F0001B6F1D6B00017DEC08F001C07CF07C5270
:1022000003E0C26BC16B656A3BEF1CF001011E6B02
:102210001F6B0001EEEC07F0700EF66E070EF76E06
:1022200021EC08F031EC08F0010E01011E6F1F6B6C
:102230000001EEEC07F07A0EF66E070EF76E21EC59
:1022400008F031EC08F0020E01011E6F1F6B000157
:10225000EEEC07F081BE0BD081BC09D082BA07D06A
:10226000860EF66E070EF76E21EC08F006D0900E83
:10227000F66E070EF76E21EC08F031EC08F0030E55
:1022800001011E6F1F6B0001EEEC07F031EC08F04E
:102290001EAC0BD001011C6B400E1B6F1D6B0001AF
:1022A0007DEC08F001C07CF00BD0110E01011C6F19
:1022B000400E1B6F1D6B00017DEC08F001C07CF02F
:1022C0007C521DE081BE1BD081BC19D082BA17D0D0
:1022D00058EC0BF00A0E3D6E3C6E866B856B86C02B
:1022E000C8F085C0C7F086C0B4F085C0B3F086C022
:1022F000BAF085C0B9F0C26BC16B1D88656A3BEF4F
:102300001CF001011E6B1F6B0001EEEC07F09A0E32
:10231000F66E070EF76E21EC08F031EC08F0010EB6
:1023200001011E6F1F6B0001EEEC07F0A40EF66EAC
:10233000070EF76E21EC08F031EC08F0020E0101F7
:102340001E6F1F6B0001EEEC07F031EC08F0030E7E
:1023500001011E6F1F6B0001EEEC07F031EC08F07D
:10236000110E01011C6F400E1B6F1D6B00017DECF7
:1023700008F001C07CF07C5213E0196AF2BE198E9D
:10238000F29E1B0E01014C6F86C04EF185C04DF1CF
:10239000010E4F6F0001AAEC01F019BEF28EFF0092
:1023A0003BEF1CF01E9201011E6B1F6B0001EEEC57
:1023B00007F0B00EF66E070EF76E050E01011D6FE9
:1023C000000195EC0BF0100EE96EC2C01EF1C1C009
:1023D0001DF1A9EC0BF031EC08F0010E01011E6FAC
:1023E0001F6B0001EEEC07F0BA0EF66E070EF76EEB
:1023F00021EC08F031EC08F0020E01011E6F1F6B9A
:102400000001EEEC07F081B007D0C60EF66E070EA5
:10241000F76E21EC08F006D0CC0EF66E070EF76EC4
:1024200021EC08F031EC08F0100E01011C6F1B6B61
:102430001D6B00017DEC08F03BEF1CF001011E6BF1
:102440001F6B0001EEEC07F0D20EF66E070EF76E72
:1024500021EC08F0010E01011E6F1F6B0001EEEC74
:1024600007F031EC08F0020E01011E6F1F6B000136
:10247000EEEC07F031EC08F0010E01011C6F110EBB
:102480001B6F1D6B00017DEC08F03BEF1CF0BE6B79
:10249000FA0EBD6FC46BC36B040E206E3C6A010163
:1024A0001E6B1F6B0001EEEC07F0E40EF66E070EDC
:1024B000F76E21EC08F031EC08F0010E01011E6FFF
:1024C0001F6B0001EEEC07F0F00EF66E070EF76ED4
:1024D00021EC08F031EC08F0020E01011E6F1F6BB9
:1024E0000001EEEC07F03A0E0101266F0001F8EC56
:1024F00007F03DC01DF1110E01011E6F000122EC1D
:102500000CF031EC08F01EAC0CD001011C6B660E17
:102510001B6F010E1D6F00017DEC08F001C07CF007
:102520000CD0110E01011C6F660E1B6F010E1D6F8A
:1025300000017DEC08F001C07CF07CBE05D07C5031
:10254000000802E2828408D07CAE02D0828604D0E9
:102550007C5202E182948296C151D10803E1C251BA
:10256000070801E0206A3BEF1CF001011E6B1F6BA6
:102570000001EEEC07F0FA0EF66E070EF76E21EC96
:1025800008F031EC08F0010E01011E6F1F6B000115
:10259000EEEC07F0090E01011B6F000163EC0CF07B
:1025A00031EC08F0020E01011E6F1F6B0001EEEC12
:1025B00007F0080EF66E080EF76E21EC08F031EC0D
:1025C00008F0110E01011C6F1B6B1D6B00017DECEF
:1025D00008F03BEF1CF001011E6B1F6B0001EEECDD
:1025E00007F0160EF66E080EF76E21EC08F031ECCF
:1025F00008F0010E01011E6F1F6B0001EEEC07F0E9
:102600000A0E01011B6F000163EC0CF031EC08F0C5
:10261000020E01011E6F1F6B0001EEEC07F0240E8D
:10262000F66E080EF76E21EC08F031EC08F0110E92
:1026300001011C6F1B6B1D6B00017DEC08F03BEF73
:102640001CF001011E6B1F6B0001EEEC07F0320E57
:10265000F66E080EF76E21EC08F031EC08F0010E72
:1026600001011E6F1F6B0001EEEC07F00B0E010164
:102670001B6F000163EC0CF031EC08F0020E01015D
:102680001E6F1F6B0001EEEC07F0400EF66E080E99
:10269000F76E21EC08F031EC08F0110E01011C6F0F
:1026A0001B6B1D6B00017DEC08F03BEF1CF0010182
:1026B0001E6B1F6B0001EEEC07F04E0EF66E080E5F
:1026C000F76E21EC08F031EC08F0010E01011E6FED
:1026D0001F6B0001EEEC07F00C0E01011B6F0001F7
:1026E00063EC0CF031EC08F0020E01011E6F1F6B61
:1026F0000001EEEC07F05C0EF66E080EF76E21ECB2
:1027000008F031EC08F0110E01011C6F1B6B1D6B02
:1027100000017DEC08F03BEF1CF001011E6B1F6B0C
:102720000001EEEC07F06C0EF66E080EF76E21EC71
:1027300008F031EC08F0010E01011E6F1F6B000163
:10274000EEEC07F00E0E01011B6F000163EC0CF0C4
:1027500031EC08F0020E01011E6F1F6B0001EEEC60
:1027600007F0760EF66E080EF76E21EC08F031ECED
:1027700008F0110E01011C6F1B6B1D6B00017DEC3D
:1027800008F03BEF1CF001011E6B1F6B0001EEEC2B
:1027900007F0860EF66E080EF76E21EC08F031ECAD
:1027A00008F0010E01011E6F1F6B0001EEEC07F037
:1027B0000D0E01011B6F000163EC0CF031EC08F011
:1027C000020E01011E6F1F6B0001EEEC07F08E0E72
:1027D000F66E080EF76E21EC08F031EC08F0110EE1
:1027E00001011C6F1B6B1D6B00017DEC08F03BEFC2
:1027F0001CF001011E6B1F6B0001EEEC07F09E0E3A
:10280000F66E080EF76E21EC08F031EC08F0010EC0
:1028100001011E6F1F6B0001EEEC07F00F0E0101AE
:102820001B6F000163EC0CF031EC08F0020E0101AB
:102830001E6F1F6B0001EEEC07F0A60EF66E080E81
:10284000F76E21EC08F031EC08F0100E01011C6F5E
:102850001B6B1D6B00017DEC08F03BEF1CF00101D0
:102860001E6B1F6B0001EEEC07F0B60EF66E080E45
:10287000F76E21EC08F031EC08F0010E01011E6F3B
:102880001F6B0001EEEC07F031EC08F0020E0101C5
:102890001E6F1F6B0001EEEC07F031EC08F0010E2B
:1028A00001011C6F110E1B6F1D6B00017DEC08F008
:1028B0003BEF1CF0BE6BFA0EBD6FC46BC36B010126
:1028C0001E6B1F6B0001EEEC07F0C40EF66E080ED7
:1028D000F76E21EC08F031EC08F0010E01011E6FDB
:1028E0001F6B0001EEEC07F00A0E01012E6F2F6B3B
:1028F00000010DEC05F00150021025E0550E01011C
:102900002E6F010E2F6F00010DEC05F002C01CF1BF
:1029100001C01BF15B0E0101266F0001F8EC07F00E
:10292000030EE96E1CC11EF11BC11DF1A9EC0BF0D9
:10293000D90EF66E080EF76E040E01011D6F000130
:1029400095EC0BF024D0B90E01012E6F010E2F6F04
:1029500000010DEC05F002C01CF101C01BF15B0E83
:102960000101266F0001F8EC07F0030EE96E1CC1AF
:102970001EF11BC11DF1A9EC0BF0E30EF66E080E63
:10298000F76E040E01011D6F000195EC0BF031ECA8
:1029900008F0020E01011E6F1F6B0001EEEC07F044
:1029A0001EAC0BD001011C6B430E1B6F1D6B000195
:1029B0007DEC08F001C07CF00BD0110E01011C6F02
:1029C000430E1B6F1D6B00017DEC08F001C07CF015
:1029D00031EC08F07CBE7FD07C500008D8B07BD0B2
:1029E00081BE79D081BC77D082BA75D0B90E010191
:1029F0002E6F010E2F6F00010DEC05F0015002103B
:102A00006AE00A0E01012E6F2F6B00010DEC05F03C
:102A10000150021010E0196AF2BE198EF29E0A0EE1
:102A200001014C6F4E6B4D6B4F6B0001AAEC01F036
:102A300019BEF28E10D0196AF2BE198EF29E0A0EDD
:102A400001014C6F4E6B010E4D6F4F6B0001AAECF4
:102A500001F019BEF28E196AF2BE198EF29E1B0E9B
:102A600001014C6F4E6B4D6B010E4F6F0001AAECD4
:102A700001F019BEF28E01011E6B1F6B0001EEEC1E
:102A800007F031EC08F0010E01011E6F1F6B000111
:102A9000EEEC07F031EC08F0020E01011E6F1F6B27
:102AA0000001EEEC07F031EC08F0030E01011E6F9F
:102AB0001F6B0001EEEC07F031EC08F00C0E010189
:102AC0001B6FFA0E1C6F0001B6EC07F001011B2F03
:102AD000F8D7FF0000017CAE03D0C26BC16B656A02
:102AE0003BEF1CF001011E6B1F6B0001EEEC07F0C9
:102AF000E80EF66E080EF76E21EC08F031EC08F0E7
:102B0000010E01011E6F1F6B0001EEEC07F07FC08C
:102B10001FF01FC01FF10A0E0101206F00010CEC15
:102B20000CF001C01BF11FC01FF10A0E0101206F44
:102B300000010CEC0CF001500A0DF3501F5C010178
:102B40001C6FF20EF66E080EF76E0C0E1D6F000174
:102B500095EC0BF01BC11DF11B0E01011E6F000156
:102B600022EC0CF02E0E0101266F0001F8EC07F0AC
:102B70001CC11DF11B0E01011E6F000122EC0CF0A7
:102B800031EC08F0020E01011E6F1F6B0001EEEC2C
:102B900007F031EC08F074520EE1510E01012E6F76
:102BA000010E2F6F00010DEC05F002C080F001C096
:102BB0007FF0010E746E110E01011C6F220E1B6F4F
:102BC000010E1D6F00017DEC08F001C07CF07C520D
:102BD00009E0020E746E036A7C50E8BE03067F268D
:102BE0000350802380AF02D0806B7F6A80BF08D003
:102BF000805303E17F50C80803E2806BC80E7F6EEC
:102C0000C151BA0803E1C2510B081CE0745002081C
:102C100016E101010BB102D0000111D0196AF2BE18
:102C2000198EF29E510E4C6F80C04EF17FC04DF157
:102C3000010E4F6F0001AAEC01F019BEF28E746A0A
:102C4000806B7F6A3BEF1CF001011E6B1F6B000164
:102C5000EEEC07F0040EF66E090EF76E21EC08F0AC
:102C600031EC08F0010E01011E6F1F6B0001EEEC4C
:102C700007F0100EF66E090EF76E0A0E01011D6FB9
:102C8000000195EC0BF0010EE96E80C01EF17FC0D3
:102C90001DF1A9EC0BF031EC08F0020E01011E6FE2
:102CA0001F6B0001EEEC07F031EC08F074520EE1FE
:102CB000530E01012E6F010E2F6F00010DEC05F078
:102CC00002C080F001C07FF0010E746E110E010190
:102CD0001C6F220E1B6F010E1D6F00017DEC08F0B2
:102CE00001C07CF07C5209E0020E746E036A7C50D5
:102CF000E8BE03067F260350802380AF02D0806B9E
:102D00007F6A80BF0CD08051020809E2FF0A03E10C
:102D10007F50E80804E2030E806FE80E7F6EC15119
:102D2000BB0803E1C2510B081CE07450020816E115
:102D300001010BB102D0000111D0196AF2BE198E47
:102D4000F29E530E4C6F80C04EF17FC04DF1010ECC
:102D50004F6F0001AAEC01F019BEF28E746A806B0D
:102D60007F6A3BEF1CF001011E6B1F6B0001EEEC54
:102D700007F0200EF66E090EF76E21EC08F031EC2C
:102D800008F0010E01011E6F1F6B0001EEEC07F051
:102D90002E0EF66E090EF76E0A0E01011D6F000170
:102DA00095EC0BF0020EE96E80C01EF17FC01DF1A4
:102DB000A9EC0BF031EC08F0020E01011E6F1F6B45
:102DC0000001EEEC07F031EC08F074520EE1550E04
:102DD00001012E6F010E2F6F00010DEC05F002C0F6
:102DE00080F001C07FF0010E746E110E01011C6FA6
:102DF000220E1B6F010E1D6F00017DEC08F001C05B
:102E00007CF07C5209E0020E746E036A7C50E8BECE
:102E100003067F260350802380AF02D0806B7F6A39
:102E200080BF08D0805303E17F50640803E2806BC9
:102E3000640E7F6EC151BC0803E1C2510B081CE057
:102E40007450020816E101010BB102D0000111D04B
:102E5000196AF2BE198EF29E550E4C6F80C04EF16B
:102E60007FC04DF1010E4F6F0001AAEC01F019BEB9
:102E7000F28E746A806B7F6A3BEF1CF001011E6B5F
:102E80001F6B0001EEEC07F03E0EF66E090EF76EBA
:102E90000A0E01011D6F000195EC0BF07FC01DF1C2
:102EA000130E01011E6F000122EC0CF05D0E0101FA
:102EB000266F0001F8EC07F031EC08F0010E01017B
:102EC0001E6F1F6B0001EEEC07F031EC08F0020EF4
:102ED00001011E6F1F6B0001EEEC07F031EC08F0F2
:102EE000110E01011C6F220E1B6F010E1D6F0001E0
:102EF0007DEC08F001C07CF07C5207E0036A7C5056
:102F0000E8BE03067F260350802380AF02D0806B8B
:102F10007F6A80BF05D08051000802E2806B7F6825
:102F2000C151BD0803E1C2510B0803E0746A7FC0C0
:102F30001FF03BEF1CF0745226E1010E746E1F501F
:102F400051080FE01F5053080CE01F50550809E0CE
:102F50001F50B50806E01F50B70803E01F50B9081E
:102F600002E11D8401D01D94000E1DB4010E01016B
:102F70001B6F1FC02EF12F6F00010DEC05F002C07A
:102F800080F001C07FF001011E6B1F6B0001EEECB1
:102F900007F04E0EF66E090EF76E030E01011D6F5F
:102FA000000195EC0BF01FC01DF1130E01011E6F07
:102FB000000122EC0CF031EC08F0010E01011E6F53
:102FC0001F6B0001EEEC07F031EC08F0020E01017E
:102FD0001E6F040E1F6F0001EEEC07F0560EF66E2A
:102FE000090EF76E060E01011D6F000195EC0BF046
:102FF000000EE96E80C01EF17FC01DF1A9EC0BF040
:103000005D0E0101266F0001F8EC07F0110E0101C1
:103010001C6F220E1B6F010E1D6F00017DEC08F06E
:1030200001C07CF07C5209E0020E746E036A7C5091
:10303000E8BE03067F260350802380AF02D0806B5A
:103040007F6A80BF07D08051000804E21DB402D01F
:10305000806B7F68C151BE0803E1C2510B0824E0B8
:10306000745002081BE101010B51030BD8A402D0DC
:10307000000114D0000E1DB4010E1B6F196AF2BEC0
:10308000198EF29E1FC04CF180C04EF17FC04DF1F1
:103090004F6F0001AAEC01F019BEF28E036A1FC047
:1030A0007FF003C080F0746A3BEF1CF001011E6BDF
:1030B0001F6B0001EEEC07F0620EF66E090EF76E64
:1030C00021EC08F031EC08F0010E01011E6F1F6BBE
:1030D0000001EEEC07F0720EF66E090EF76E21ECB1
:1030E00008F031EC08F0020E01011E6F1F6B0001A9
:1030F000EEEC07F031EC08F0110E01011C6F400EF0
:103100001B6F1D6B00017DEC08F001C07CF07C5250
:1031100005E01F6A0B0EC26FC10EC16FACD3010177
:103120001E6B1F6B0001EEEC07F0800EF66E090EB1
:10313000F76E21EC08F031EC08F0010E01011E6F72
:103140001F6B0001EEEC07F0900EF66E090EF76EA5
:1031500021EC08F031EC08F0020E01011E6F1F6B2C
:103160000001EEEC07F031EC08F0100E01011C6FCD
:10317000400E1B6F1D6B00017DEC08F001C07CF060
:103180007C5206E0010E1F6E0B0EC26FC10EC16FA6
:1031900072D301010BAF4DD1196AF2BE198EF29EA6
:1031A0004C6B4E6B0C0E4D6F4F6B0001AAEC01F097
:1031B00019BEF28E1F5211E1196AF2BE198EF29EEB
:1031C000010E01014C6F4E6B390E4D6F4F6B0001BC
:1031D000AAEC01F019BEF28E12D01F2C10D0196A81
:1031E000F2BE198EF29E010E01014C6F4E6B340E31
:1031F0004D6F4F6B0001AAEC01F019BEF28E196AF7
:10320000F2BE198EF29E020E01014C6F4E6B100E33
:103210004D6F4F6B0001AAEC01F019BEF28E1F52E8
:1032200011E1196AF2BE198EF29E030E01014C6F74
:103230004E6B360E4D6F4F6B0001AAEC01F019BEBC
:10324000F28E12D01F2C10D0196AF2BE198EF29E87
:10325000030E01014C6F4E6B300E4D6F4F6B000132
:10326000AAEC01F019BEF28E196AF2BE198EF29E16
:10327000040E01014C6F4E6B140E4D6F4F6B00012D
:10328000AAEC01F019BEF28E1F5211E1196AF2BECA
:10329000198EF29E050E01014C6F4E6B320E4D6F72
:1032A0004F6B0001AAEC01F019BEF28E12D01F2C58
:1032B00010D0196AF2BE198EF29E050E01014C6FF4
:1032C0004E6B2C0E4D6F4F6B0001AAEC01F019BE36
:1032D000F28E196AF2BE198EF29E060E01014C6F33
:1032E0004E6B020E4D6F4F6B0001AAEC01F019BE40
:1032F000F28E196AF2BE198EF29E070E01014C6F12
:103300004E6B010E4D6F4F6B0001AAEC01F019BE20
:10331000F28E196AF2BE198EF29E080E01014C6FF0
:103320004E6B040E4D6F4F6B0001AAEC01F019BEFD
:10333000F28E1F5211E1196AF2BE198EF29E090E29
:1033400001014C6F4E6B320E4D6F4F6B0001AAECBA
:1033500001F019BEF28E12D01F2C10D0196AF2BEE5
:10336000198EF29E090E01014C6F4E6B2C0E4D6FA3
:103370004F6B0001AAEC01F019BEF28E1F5212E150
:10338000196AF2BE198EF29E510E01014C6F4E6BFE
:10339000470E4D6F010E4F6F0001AAEC01F019BEF0
:1033A000F28E13D01F2C11D0196AF2BE198EF29E24
:1033B000510E01014C6F4E6B3E0E4D6F010E4F6F63
:1033C0000001AAEC01F019BEF28E196AF2BE198E44
:1033D000F29E530E01014C6F010E4E6F9C0E4D6F0D
:1033E000010E4F6F0001AAEC01F019BEF28E196AAE
:1033F000F2BE198EF29E550E01014C6F4E6B280ED7
:103400004D6F010E4F6F0001AAEC01F019BEF28E54
:10341000196AF2BE198EF29E590E01014C6F4E6B65
:10342000080E4D6F4F6B0001AAEC01F019BEF28E31
:1034300001010B0E0001C26FBC0EC16F1CD2010155
:103440001E6B1F6B0001EEEC07F09E0EF66E090E70
:10345000F76E21EC08F031EC08F0010E01011E6F4F
:103460001F6B0001EEEC07F031EC08F0020E0101D9
:103470001E6F1F6B0001EEEC07F031EC08F001014C
:103480001C6B110E1B6F1D6B00017DEC08F0F3D15E
:1034900001011E6B1F6B0001EEEC07F0A60EF66E2D
:1034A000090EF76E21EC08F031EC08F0010E010175
:1034B0001E6F1F6B0001EEEC07F031EC08F0020EFE
:1034C00001011E6F1F6B0001EEEC07F031EC08F0FC
:1034D000010E696E695006080BE3036A69500B0F11
:1034E000E96E010E0320EA6E300EEF6E692AF2D704
:1034F000010E01011C6F100E1B6F1D6B00017DEC96
:1035000008F0B9D1C4EC0CF0110E01011C6F220EB1
:103510001B6F010E1D6F00017DEC08F001C07CF0F7
:103520007CBE2BD07C50000828E2880EC15D0101D2
:103530001B6F130E0001C25901011C6F0B0E1B25DE
:10354000E96E010E1C21EA6EEF503808D8B002D0A7
:10355000000113D0880E0001C15D01011B6F130E25
:103560000001C25901011C6F0B0E1B25E96E010EF3
:103570001C21EA6EEF2A29D000017CAE27D0880EEC
:10358000C15D01011B6F130E0001C25901011C6FC7
:103590000B0E1B25E96E010E1C21EA6EEF50300860
:1035A000D8A002D0000112D0880E0001C15D010137
:1035B0001B6F130E0001C25901011C6F0B0E1B255E
:1035C000E96E010E1C21EA6EEF06000154D1C4EC35
:1035D0000CF0140E01011C6F220E1B6F010E1D6FEB
:1035E00000017DEC08F001C07CF07CBE2BD07C504B
:1035F000000828E2880EC15D01011B6F130E000157
:10360000C25901011C6F0B0E1B25E96E010E1C2116
:10361000EA6EEF503808D8B002D0000113D0880EFF
:103620000001C15D01011B6F130E0001C2590101B0
:103630001C6F0B0E1B25E96E010E1C21EA6EEF2A92
:1036400029D000017CAE27D0880EC15D01011B6F1F
:10365000130E0001C25901011C6F0B0E1B25E96EF0
:10366000010E1C21EA6EEF503008D8A002D00001F4
:1036700012D0880E0001C15D01011B6F130E000105
:10368000C25901011C6F0B0E1B25E96E010E1C2196
:10369000EA6EEF060001EFD0010EEA6E120EE96E3F
:1036A000000E6FEC00F00A000900F550EE6E000904
:1036B000FBE1010E01011C6F0C0E1B6F010E1E6F52
:1036C000120E1D6F206B060E1F6F000116EC0DF021
:1036D000015204E1FF0E01010B130001010EEA6E1D
:1036E000120EE96E000E7BEC00F00A000900F550A6
:1036F000EE6E0009FBE1010E01011C6F0C0E1B6F49
:10370000010E1E6F120E1D6F206B060E1F6F000143
:1037100016EC0DF0015204E1030E01010B13000140
:10372000010EEA6E120EE96E000E87EC00F00A0040
:103730000900F550EE6E0009FBE1010E01011C6F5E
:103740000C0E1B6F010E1E6F120E1D6F206B060EEE
:103750001F6F000116EC0DF0015203E101010B8116
:10376000000101010B5343E01E6B1F6B0001EEECE7
:1037700007F0B00EF66E090EF76E21EC08F031EC92
:1037800008F0010E01011E6F1F6B0001EEEC07F047
:10379000BE0EF66E090EF76E21EC08F031EC08F063
:1037A000020E01011E6F1F6B0001EEEC07F0C80E48
:1037B000F66E090EF76E21EC08F0200E0101266F5F
:1037C0000001F8EC07F0460E0101266F0001F8EC4D
:1037D00007F0100EE96E0A0E01011E6F3C0E1D6F00
:1037E0000001A9EC0BF031EC08F020D001011E6BB8
:1037F0001F6B0001EEEC07F031EC08F0010E010147
:103800001E6F1F6B0001EEEC07F0D20EF66E090E74
:10381000F76E21EC08F031EC08F0020E01011E6F8A
:103820001F6B0001EEEC07F031EC08F0140E010103
:103830001C6F1B6B1D6B00017DEC08F01CD001019F
:103840001C6B030E1B6F1D6B00017DEC08F001C0AB
:103850007CF0C46BC36B7C520BE0C26BC16B206A03
:10386000656AC46BC80EC36F7B6A0A0E3D6E3C6E00
:1038700002D0C26BC16B79D0C151C211D8A475D02E
:103880001DA673D01D961EA804D06E5201E11E988D
:1038900017D06E5215E06E5009080AE1C26BC16B79
:1038A000206A656A1E9CC46BC80EC36F746A04D01C
:1038B000030EC26FE80EC16F1E88C46BC36B746ABF
:1038C000BD51BE1152E0C151C2114FE101011E6B49
:1038D0001F6B0001EEEC07F0E00EF66E090EF76EBE
:1038E000070E01011D6F000195EC0BF0010EE96E52
:1038F00086C01EF185C01DF1A9EC0BF031EC08F07B
:10390000010E01011E6F1F6B0001EEEC07F0EC0EC3
:10391000F66E090EF76E21EC08F0020E01011E6F23
:103920001F6B0001EEEC07F0FE0EF66E090EF76E4F
:10393000050E01011D6F000195EC0BF03DC01DF15E
:10394000110E01011E6F000122EC0CF031EC08F0A9
:10395000030E01011E6F1F6B0001EEEC07F0080E55
:10396000F66E0A0EF76E21EC08F020500AE0040A09
:10397000D8B454D1010AD8B452D10D0AD8B473D1F5
:103980009CD11DA205D11D92BAC0BCF0B9C0BBF03C
:1039900077C07AF08551B95D03E18651BA5D05E0E3
:1039A00086C0BAF085C0B9F0F5D73D50775C03E02A
:1039B0003DC077F0FAD7BA51EA08D8A0E9D004E1BF
:1039C000B9515F08D8A0E4D0BA51B45D09E303E16E
:1039D000B351B95D05E21EA401D01D981E8409D023
:1039E000B451BA5D06E303E1B951B35D02E21D884B
:1039F0001E94196AF2BE198EF29EBAC04DF1B9C07A
:103A00004CF188C04FF187C04EF1CEEC00F019BEEA
:103A1000F28E02C01CF101C01BF1010101A017D000
:103A2000196AF2BE198EF29EBAC04DF1B9C04CF1BE
:103A300088C04FF187C04EF10001CEEC00F019BEF6
:103A4000F28E00C0B5F003C0B6F018D00101196ABB
:103A5000F2BE198EF29EBAC04DF1B9C04CF188C0C9
:103A60004FF187C04EF10001CEEC00F019BEF28E8E
:103A70000050875DB56F03508859B66FB6C02EF100
:103A8000B5C02DF10101306B640E2F6F0001B6EC53
:103A900005F002C01CF101C01BF1196AF2BE198EBB
:103AA000F29E02C04DF101C04CF1B2C04FF1B1C065
:103AB0004EF1CEEC00F019BEF28E01C01BF10A0EE1
:103AC00001010124016E000E022001C04BF01DA86F
:103AD00041D04B50425C07E243504B5C04E21D8AEC
:103AE0004BC03CF036D04B50405C07E377500A089F
:103AF00002E00A0E3C6E1D9A2CD04B50405C0FE247
:103B00004B50425C0CE31DAA03D04BC03CF006D0E6
:103B1000020E425C4B5C02E344C03CF01AD04150C0
:103B20004B5C10E243504B5C0DE31DAA03D04BC02D
:103B30003CF007D0020E43244B5C01E002E245C09A
:103B40003CF007D041504B5C04E30A0E4A243C6E23
:103B50001D9A02D04BC03CF03C50775C1B6F1B5150
:103B60001BAF03D0000ED8801B55006EE8BE0BD0F3
:103B70000050475C08E23C50775C03E28296828406
:103B800002D082948286BAC0B4F0B9C0B3F000010A
:103B90001DA043D01D9081B207D0232A23500308D3
:103BA00002E2050E206E01D0236A1EAE08D01E9ED2
:103BB0001EBA05D01D9C080E206E020E7B6E010100
:103BC0000BA109D0652C07D00001BE6BFA0EBD6FAA
:103BD000C46BC36B01010001BA51EA0806E303E1BB
:103BE000B9515F0802E363EC0DF084C063F083C059
:103BF00064F01EB212D0B951C75D01011B6F1B5199
:103C00001BAF03D0000ED8801B55006EE8BE04D059
:103C10000050040801E21E82000150D04FD01DA0C8
:103C200021D01D90BA51EA0806E303E1B9515F08BB
:103C300002E363EC0DF084C063F083C064F02350B2
:103C40000C0803E3232A82860DD0829681A208D035
:103C5000232A2350100803E21E8E206A236A02D012
:103C60000D0E236E2BD01DA002D01D907B067B5223
:103C700023E1050E7B6E1EB61FD058EC0BF0120E22
:103C80004A243D5C01E018E258EC0BF0120E4A2485
:103C90003D5C01E011E20A0E3D6E3C6E206AC26B93
:103CA000C16B656AC46BC80EC36FBE6BBD6B86C04B
:103CB000BAF085C0B9F07B6A01D0206A75EF0FF0C9
:023CC0000300FF
:0200000400F00A
:1000000000000000000000000000000000000000F0
:1000100000000000000000000000000000000000E0
:1000200000000000000000000000000000000000D0
:1000300000000000000000000000000000000000C0
:1000400000000000000000000000000000000000B0
:1000500000000000000000000000000000000000A0
:100060000000000000000000000000000000000090
:100070000000000000000000000000000000000080
:020000040030CA
:0E00000000C21E150087810000800FE00F4037
:00000001FF
